:0200000480007A
:100000006F00C004732F2034930F8000630AFF0336
:10001000930F90006306FF03930FB0006302FF038A
:10002000170F0080130F0FFE63040F0067000F000F
:10003000732F203463540F006F004000136E9E53E3
:10004000171F00002320CFFD6FF09FFF732540F1A5
:100050006310050073251030635805000F00F00F82
:10006000130E100073000000130E00009702000032
:10007000938282F973905230735020307350303035
:1000800073504030970200809382C2F7638C020065
:10009000739052109302B01A739022307323203061
:1000A000E39E62F873500030970200009382420191
:1000B00073901234732540F173002030130E20002A
:1000C000930000001301000063F620006312C035A6
:1000D0006316C001E3FE20FE631CC033130E300024
:1000E000930010001301100063F620006312C03368
:1000F0006316C001E3FE20FE631CC031130E4000F6
:100100009300F0FF1301F0FF63F620006312C0318B
:100110006316C001E3FE20FE631CC02F130E5000C7
:10012000930010001301000063F620006312C02F3B
:100130006316C001E3FE20FE631CC02D130E600099
:100140009300F0FF1301E0FF63F620006312C02D5F
:100150006316C001E3FE20FE631CC02B130E70006B
:100160009300F0FF1301000063F620006312C02B20
:100170006316C001E3FE20FE631CC029130E80003D
:10018000930000001301100063F420006314C00109
:100190006310C029E3FE20FE130E90009300E0FFE1
:1001A0001301F0FF63F420006314C0016312C02741
:1001B000E3FE20FE130EA000930000001301F0FFE9
:1001C00063F420006314C0016314C025E3FE20FE25
:1001D000130EB000B70000809380F0FF370100805D
:1001E00063F420006314C0016314C023E3FE20FE07
:1001F000130EC00013020000B70000F09380F0FF60
:10020000370100F063F62020130212009302200051
:10021000E31452FE130ED00013020000B70000F0EA
:100220009380F0FF370100F01300000063F2201EFE
:100230001302120093022000E31252FE130EE0009C
:1002400013020000B70000F09380F0FF370100F0C8
:10025000130000001300000063FC201A13021200B8
:1002600093022000E31052FE130EF0001302000070
:10027000B70000F09380F0FF13000000370100F09A
:1002800063F820181302120093022000E31252FEBA
:10029000130E000113020000B70000F09380F0FF7E
:1002A00013000000370100F01300000063F2201675
:1002B0001302120093022000E31052FE130E1001ED
:1002C00013020000B70000F09380F0FF130000005D
:1002D00013000000370100F063FC2012130212002B
:1002E00093022000E31052FE130E200113020000BF
:1002F000B70000F09380F0FF370100F063FA2010A0
:100300001302120093022000E31452FE130E300178
:1003100013020000B70000F09380F0FF370100F0F7
:100320001300000063F6200E130212009302200057
:10033000E31252FE130E400113020000B70000F05A
:100340009380F0FF370100F013000000130000005D
:1003500063F0200C1302120093022000E31052FEFF
:10036000130E500113020000B70000F09380F0FF5D
:1003700013000000370100F063FC20081302120094
:1003800093022000E31252FE130E600113020000DC
:10039000B70000F09380F0FF13000000370100F079
:1003A0001300000063F620061302120093022000DF
:1003B000E31052FE130E700113020000B70000F0AC
:1003C0009380F0FF1300000013000000370100F0DD
:1003D00063F020041302120093022000E31052FE87
:1003E0009300100063FA00009380100093801000C7
:1003F0009380100093801000938010009380100071
:10040000930E3000130E80016394D001631CC00171
:100410000F00F00F63000E00131E1E00136E1E006F
:10042000730000000F00F00F130E100073000000A7
:10043000731000C000000000000000000000000079
:0404400000000000B8
:1010000000000000000000000000000000000000E0
:1010100000000000000000000000000000000000D0
:1010200000000000000000000000000000000000C0
:1010300000000000000000000000000000000000B0
:081040000000000000000000A8
:040000058000200057
:00000001FF
